 jmap

 Timestamp is 68fa9022 (Thu Oct 23 20:29:22 2025)

 Preferred load address is 00400000

 Start         Length     Name                   Class
 0001:00000000 00000dc4H .text$mn                CODE
 0002:00000000 000000e8H .idata$5                DATA
 0002:000000e8 00000008H .00cfg                  DATA
 0002:000000f0 00000004H .CRT$XCA                DATA
 0002:000000f4 00000004H .CRT$XCAA               DATA
 0002:000000f8 00000004H .CRT$XCZ                DATA
 0002:000000fc 00000004H .CRT$XIA                DATA
 0002:00000100 00000004H .CRT$XIAA               DATA
 0002:00000104 00000004H .CRT$XIAC               DATA
 0002:00000108 00000004H .CRT$XIZ                DATA
 0002:0000010c 00000004H .CRT$XPA                DATA
 0002:00000110 00000004H .CRT$XPZ                DATA
 0002:00000114 00000004H .CRT$XTA                DATA
 0002:00000118 00000008H .CRT$XTZ                DATA
 0002:0000011c 00000000H .gfids$y                DATA
 0002:00000120 00000260H .rdata                  DATA
 0002:00000380 00000000H .rdata$CastGuardVftablesA DATA
 0002:00000380 00000000H .rdata$CastGuardVftablesC DATA
 0002:00000380 00000004H .rdata$sxdata           DATA
 0002:00000384 00000064H .rdata$voltmd           DATA
 0002:000003e8 00000314H .rdata$zzzdbg           DATA
 0002:000006fc 00000004H .rtc$IAA                DATA
 0002:00000700 00000004H .rtc$IZZ                DATA
 0002:00000704 00000004H .rtc$TAA                DATA
 0002:00000708 00000008H .rtc$TZZ                DATA
 0002:00000710 0000003cH .xdata$x                DATA
 0002:0000074c 00000000H .edata                  DATA
 0002:0000074c 000000b4H .idata$2                DATA
 0002:00000800 00000014H .idata$3                DATA
 0002:00000814 000000e8H .idata$4                DATA
 0002:000008fc 000004c2H .idata$6                DATA
 0003:00000000 00000040H .data                   DATA
 0003:00000040 00000378H .bss                    DATA
 0004:00000000 00000060H .rsrc$01                DATA
 0004:00000060 00000330H .rsrc$02                DATA

  Address         Publics by Value              Rva+Base       Lib:Object

 0000:00000000       ___AbsoluteZero            00000000     <absolute>
 0000:00000000       ___arm64x_extra_rfe_table  00000000     <absolute>
 0000:00000000       ___arm64x_extra_rfe_table_size 00000000     <absolute>
 0000:00000000       ___arm64x_native_entrypoint 00000000     <absolute>
 0000:00000000       ___arm64x_redirection_metadata 00000000     <absolute>
 0000:00000000       ___arm64x_redirection_metadata_count 00000000     <absolute>
 0000:00000000       ___dynamic_value_reloc_table 00000000     <absolute>
 0000:00000000       ___enclave_config          00000000     <absolute>
 0000:00000000       ___guard_check_icall_a64n_fptr 00000000     <absolute>
 0000:00000000       ___guard_eh_cont_count     00000000     <absolute>
 0000:00000000       ___guard_eh_cont_table     00000000     <absolute>
 0000:00000000       ___guard_fids_count        00000000     <absolute>
 0000:00000000       ___guard_fids_table        00000000     <absolute>
 0000:00000000       ___guard_iat_count         00000000     <absolute>
 0000:00000000       ___guard_iat_table         00000000     <absolute>
 0000:00000000       ___guard_longjmp_count     00000000     <absolute>
 0000:00000000       ___guard_longjmp_table     00000000     <absolute>
 0000:00000000       ___hybrid_auxiliary_delayload_iat 00000000     <absolute>
 0000:00000000       ___hybrid_auxiliary_delayload_iat_copy 00000000     <absolute>
 0000:00000000       ___hybrid_auxiliary_iat    00000000     <absolute>
 0000:00000000       ___hybrid_auxiliary_iat_copy 00000000     <absolute>
 0000:00000000       ___hybrid_code_map         00000000     <absolute>
 0000:00000000       ___hybrid_code_map_count   00000000     <absolute>
 0000:00000000       ___hybrid_image_info_bitfield 00000000     <absolute>
 0000:00000000       ___x64_code_ranges_to_entry_points 00000000     <absolute>
 0000:00000000       ___x64_code_ranges_to_entry_points_count 00000000     <absolute>
 0000:00000001       ___safe_se_handler_count   00000001     <absolute>
 0000:00000100       ___guard_flags             00000100     <absolute>
 0000:00000000       ___ImageBase               00400000     <linker-defined>
 0001:00000000       ___local_stdio_printf_options 00401000 f i main.obj
 0001:00000006       __vfprintf_l               00401006 f i main.obj
 0001:0000002a       _main                      0040102a f   main.obj
 0001:00000101       _printf                    00401101 f i main.obj
 0001:0000011f       _JLI_MemAlloc              0040111f f   jli:jli.dll
 0001:00000125       _JLI_GetStdArgs            00401125 f   jli:jli.dll
 0001:0000012b       _JLI_GetStdArgc            0040112b f   jli:jli.dll
 0001:00000131       _JLI_CmdToArgs             00401131 f   jli:jli.dll
 0001:00000137       _JLI_Launch                00401137 f   jli:jli.dll
 0001:00000384       _mainCRTStartup            00401384 f   MSVCRT:exe_main.obj
 0001:000003d2       ___scrt_acquire_startup_lock 004013d2 f   MSVCRT:utility.obj
 0001:00000404       ___scrt_initialize_crt     00401404 f   MSVCRT:utility.obj
 0001:0000043d       ___scrt_initialize_onexit_tables 0040143d f   MSVCRT:utility.obj
 0001:000004c4       ___scrt_is_nonwritable_in_current_image 004014c4 f   MSVCRT:utility.obj
 0001:00000558       ___scrt_release_startup_lock 00401558 f   MSVCRT:utility.obj
 0001:00000575       ___scrt_uninitialize_crt   00401575 f   MSVCRT:utility.obj
 0001:0000059d       __onexit                   0040159d f   MSVCRT:utility.obj
 0001:000005ca       _atexit                    004015ca f   MSVCRT:utility.obj
 0001:0000062c       ___security_init_cookie    0040162c f   MSVCRT:gs_support.obj
 0001:00000677       ___scrt_exe_initialize_mta 00401677 f   MSVCRT:utility_desktop.obj
 0001:00000677       ___scrt_initialize_winrt   00401677 f   MSVCRT:utility_desktop.obj
 0001:00000677       ___scrt_stub_for_initialize_mta 00401677 f   MSVCRT:utility_desktop.obj
 0001:00000677       __get_startup_commit_mode  00401677 f   MSVCRT:commit_mode.obj
 0001:00000677       __get_startup_new_mode     00401677 f   MSVCRT:new_mode.obj
 0001:00000677       __get_startup_thread_locale_mode 00401677 f   MSVCRT:thread_locale.obj
 0001:00000677       __matherr                  00401677 f   MSVCRT:matherr.obj
 0001:0000067a       __get_startup_argv_mode    0040167a f   MSVCRT:argv_mode.obj
 0001:0000067e       __get_startup_file_mode    0040167e f   MSVCRT:file_mode.obj
 0001:00000684       ?__scrt_initialize_type_info@@YAXXZ 00401684 f   MSVCRT:tncleanup.obj
 0001:00000690       ___acrt_initialize         00401690 f   MSVCRT:ucrt_stubs.obj
 0001:00000690       ___acrt_uninitialize       00401690 f   MSVCRT:ucrt_stubs.obj
 0001:00000690       ___scrt_stub_for_acrt_initialize 00401690 f   MSVCRT:ucrt_stubs.obj
 0001:00000690       ___scrt_stub_for_acrt_uninitialize 00401690 f   MSVCRT:ucrt_stubs.obj
 0001:00000690       ___vcrt_initialize         00401690 f   MSVCRT:ucrt_stubs.obj
 0001:00000690       ___vcrt_uninitialize       00401690 f   MSVCRT:ucrt_stubs.obj
 0001:00000690       __should_initialize_environment 00401690 f   MSVCRT:env_mode.obj
 0001:00000693       __initialize_default_precision 00401693 f   MSVCRT:default_precision.obj
 0001:000006b4       @_guard_check_icall_nop@4  004016b4 f   MSVCRT:guard_support.obj
 0001:000006b4       __initialize_denormal_control 004016b4 f   MSVCRT:denormal_control.obj
 0001:000006b4       __initialize_invalid_parameter_handler 004016b4 f   MSVCRT:invalid_parameter_handler.obj
 0001:000006b7       ___local_stdio_scanf_options 004016b7 f i MSVCRT:default_local_stdio_options.obj
 0001:000006bd       ___scrt_initialize_default_local_stdio_options 004016bd f   MSVCRT:default_local_stdio_options.obj
 0001:000006da       ___scrt_is_user_matherr_present 004016da f   MSVCRT:matherr_detection.obj
 0001:000006e6       ___scrt_get_dyn_tls_init_callback 004016e6 f   MSVCRT:dyn_tls_init.obj
 0001:000006ec       ___scrt_get_dyn_tls_dtor_callback 004016ec f   MSVCRT:dyn_tls_dtor.obj
 0001:000006f2       ___scrt_fastfail           004016f2 f   MSVCRT:utility_desktop.obj
 0001:0000080d       ___scrt_initialize_mta     0040180d f   MSVCRT:utility_desktop.obj
 0001:00000812       ___scrt_is_managed_app     00401812 f   MSVCRT:utility_desktop.obj
 0001:00000854       ___scrt_set_unhandled_exception_filter 00401854 f   MSVCRT:utility_desktop.obj
 0001:00000860       ___scrt_unhandled_exception_filter@4 00401860 f   MSVCRT:utility_desktop.obj
 0001:000008b6       __crt_debugger_hook        004018b6 f   MSVCRT:utility_desktop.obj
 0001:000008be       __RTC_Initialize           004018be f   MSVCRT:initsect.obj
 0001:000008ea       __RTC_Terminate            004018ea f   MSVCRT:initsect.obj
 0001:00000920       __SEH_prolog4              00401920 f   MSVCRT:sehprolg4.obj
 0001:00000965       __except_handler4          00401965 f   MSVCRT:chandler4gs.obj
 0001:00000994       ___isa_available_init      00401994 f   MSVCRT:cpu_disp.obj
 0001:00000b68       ___scrt_is_ucrt_dll_in_use 00401b68 f   MSVCRT:ucrt_detection.obj
 0001:00000b74       @__security_check_cookie@4 00401b74 f   MSVCRT:secchk.obj
 0001:00000b82       ___raise_securityfailure   00401b82 f   MSVCRT:gs_report.obj
 0001:00000baa       ___report_gsfailure        00401baa f   MSVCRT:gs_report.obj
 0001:00000ca4       ___current_exception       00401ca4 f   vcruntime:VCRUNTIME140.dll
 0001:00000caa       ___current_exception_context 00401caa f   vcruntime:VCRUNTIME140.dll
 0001:00000cb0       _memset                    00401cb0 f   vcruntime:VCRUNTIME140.dll
 0001:00000cb6       __except_handler4_common   00401cb6 f   vcruntime:VCRUNTIME140.dll
 0001:00000cbc       ___p___argc                00401cbc f   ucrt:api-ms-win-crt-runtime-l1-1-0.dll
 0001:00000cc2       ___p___argv                00401cc2 f   ucrt:api-ms-win-crt-runtime-l1-1-0.dll
 0001:00000cc8       __seh_filter_exe           00401cc8 f   ucrt:api-ms-win-crt-runtime-l1-1-0.dll
 0001:00000cce       __set_app_type             00401cce f   ucrt:api-ms-win-crt-runtime-l1-1-0.dll
 0001:00000cd4       ___setusermatherr          00401cd4 f   ucrt:api-ms-win-crt-math-l1-1-0.dll
 0001:00000cda       __configure_narrow_argv    00401cda f   ucrt:api-ms-win-crt-runtime-l1-1-0.dll
 0001:00000ce0       __initialize_narrow_environment 00401ce0 f   ucrt:api-ms-win-crt-runtime-l1-1-0.dll
 0001:00000ce6       __get_initial_narrow_environment 00401ce6 f   ucrt:api-ms-win-crt-runtime-l1-1-0.dll
 0001:00000cec       __initterm                 00401cec f   ucrt:api-ms-win-crt-runtime-l1-1-0.dll
 0001:00000cf2       __initterm_e               00401cf2 f   ucrt:api-ms-win-crt-runtime-l1-1-0.dll
 0001:00000cf8       _exit                      00401cf8 f   ucrt:api-ms-win-crt-runtime-l1-1-0.dll
 0001:00000cfe       __exit                     00401cfe f   ucrt:api-ms-win-crt-runtime-l1-1-0.dll
 0001:00000d04       __set_fmode                00401d04 f   ucrt:api-ms-win-crt-stdio-l1-1-0.dll
 0001:00000d0a       __cexit                    00401d0a f   ucrt:api-ms-win-crt-runtime-l1-1-0.dll
 0001:00000d10       __c_exit                   00401d10 f   ucrt:api-ms-win-crt-runtime-l1-1-0.dll
 0001:00000d16       __register_thread_local_exe_atexit_callback 00401d16 f   ucrt:api-ms-win-crt-runtime-l1-1-0.dll
 0001:00000d1c       __configthreadlocale       00401d1c f   ucrt:api-ms-win-crt-locale-l1-1-0.dll
 0001:00000d22       __set_new_mode             00401d22 f   ucrt:api-ms-win-crt-heap-l1-1-0.dll
 0001:00000d28       ___p__commode              00401d28 f   ucrt:api-ms-win-crt-stdio-l1-1-0.dll
 0001:00000d2e       __initialize_onexit_table  00401d2e f   ucrt:api-ms-win-crt-runtime-l1-1-0.dll
 0001:00000d34       __register_onexit_function 00401d34 f   ucrt:api-ms-win-crt-runtime-l1-1-0.dll
 0001:00000d3a       __crt_atexit               00401d3a f   ucrt:api-ms-win-crt-runtime-l1-1-0.dll
 0001:00000d40       __controlfp_s              00401d40 f   ucrt:api-ms-win-crt-runtime-l1-1-0.dll
 0001:00000d46       _terminate                 00401d46 f   ucrt:api-ms-win-crt-runtime-l1-1-0.dll
 0001:00000d4c       __filter_x86_sse2_floating_point_exception 00401d4c f   MSVCRT:x86_exception_filter.obj
 0001:00000d4c       __filter_x86_sse2_floating_point_exception_default 00401d4c f   MSVCRT:x86_exception_filter.obj
 0002:00000000       __imp__IsDebuggerPresent@0 00402000     kernel32:KERNEL32.dll
 0002:00000004       __imp__GetCurrentProcess@0 00402004     kernel32:KERNEL32.dll
 0002:00000008       __imp__GetModuleHandleW@4  00402008     kernel32:KERNEL32.dll
 0002:0000000c       __imp__IsProcessorFeaturePresent@4 0040200c     kernel32:KERNEL32.dll
 0002:00000010       __imp__SetUnhandledExceptionFilter@4 00402010     kernel32:KERNEL32.dll
 0002:00000014       __imp__GetCommandLineA@0   00402014     kernel32:KERNEL32.dll
 0002:00000018       __imp__QueryPerformanceCounter@4 00402018     kernel32:KERNEL32.dll
 0002:0000001c       __imp__GetCurrentProcessId@0 0040201c     kernel32:KERNEL32.dll
 0002:00000020       __imp__GetCurrentThreadId@0 00402020     kernel32:KERNEL32.dll
 0002:00000024       __imp__GetSystemTimeAsFileTime@4 00402024     kernel32:KERNEL32.dll
 0002:00000028       __imp__InitializeSListHead@4 00402028     kernel32:KERNEL32.dll
 0002:0000002c       __imp__UnhandledExceptionFilter@4 0040202c     kernel32:KERNEL32.dll
 0002:00000030       __imp__TerminateProcess@8  00402030     kernel32:KERNEL32.dll
 0002:00000034       \177KERNEL32_NULL_THUNK_DATA 00402034     kernel32:KERNEL32.dll
 0002:00000038       __imp____current_exception 00402038     vcruntime:VCRUNTIME140.dll
 0002:0000003c       __imp____current_exception_context 0040203c     vcruntime:VCRUNTIME140.dll
 0002:00000040       __imp___except_handler4_common 00402040     vcruntime:VCRUNTIME140.dll
 0002:00000044       __imp__memset              00402044     vcruntime:VCRUNTIME140.dll
 0002:00000048       \177VCRUNTIME140_NULL_THUNK_DATA 00402048     vcruntime:VCRUNTIME140.dll
 0002:0000004c       __imp__getenv              0040204c     ucrt:api-ms-win-crt-environment-l1-1-0.dll
 0002:00000050       \177api-ms-win-crt-environment-l1-1-0_NULL_THUNK_DATA 00402050     ucrt:api-ms-win-crt-environment-l1-1-0.dll
 0002:00000054       __imp___set_new_mode       00402054     ucrt:api-ms-win-crt-heap-l1-1-0.dll
 0002:00000058       \177api-ms-win-crt-heap-l1-1-0_NULL_THUNK_DATA 00402058     ucrt:api-ms-win-crt-heap-l1-1-0.dll
 0002:0000005c       __imp___configthreadlocale 0040205c     ucrt:api-ms-win-crt-locale-l1-1-0.dll
 0002:00000060       \177api-ms-win-crt-locale-l1-1-0_NULL_THUNK_DATA 00402060     ucrt:api-ms-win-crt-locale-l1-1-0.dll
 0002:00000064       __imp____setusermatherr    00402064     ucrt:api-ms-win-crt-math-l1-1-0.dll
 0002:00000068       \177api-ms-win-crt-math-l1-1-0_NULL_THUNK_DATA 00402068     ucrt:api-ms-win-crt-math-l1-1-0.dll
 0002:0000006c       __imp____p___argv          0040206c     ucrt:api-ms-win-crt-runtime-l1-1-0.dll
 0002:00000070       __imp___seh_filter_exe     00402070     ucrt:api-ms-win-crt-runtime-l1-1-0.dll
 0002:00000074       __imp___set_app_type       00402074     ucrt:api-ms-win-crt-runtime-l1-1-0.dll
 0002:00000078       __imp____p___argc          00402078     ucrt:api-ms-win-crt-runtime-l1-1-0.dll
 0002:0000007c       __imp___controlfp_s        0040207c     ucrt:api-ms-win-crt-runtime-l1-1-0.dll
 0002:00000080       __imp___configure_narrow_argv 00402080     ucrt:api-ms-win-crt-runtime-l1-1-0.dll
 0002:00000084       __imp__terminate           00402084     ucrt:api-ms-win-crt-runtime-l1-1-0.dll
 0002:00000088       __imp___get_initial_narrow_environment 00402088     ucrt:api-ms-win-crt-runtime-l1-1-0.dll
 0002:0000008c       __imp___initterm           0040208c     ucrt:api-ms-win-crt-runtime-l1-1-0.dll
 0002:00000090       __imp___initterm_e         00402090     ucrt:api-ms-win-crt-runtime-l1-1-0.dll
 0002:00000094       __imp__exit                00402094     ucrt:api-ms-win-crt-runtime-l1-1-0.dll
 0002:00000098       __imp___exit               00402098     ucrt:api-ms-win-crt-runtime-l1-1-0.dll
 0002:0000009c       __imp___crt_atexit         0040209c     ucrt:api-ms-win-crt-runtime-l1-1-0.dll
 0002:000000a0       __imp___cexit              004020a0     ucrt:api-ms-win-crt-runtime-l1-1-0.dll
 0002:000000a4       __imp___register_thread_local_exe_atexit_callback 004020a4     ucrt:api-ms-win-crt-runtime-l1-1-0.dll
 0002:000000a8       __imp___initialize_narrow_environment 004020a8     ucrt:api-ms-win-crt-runtime-l1-1-0.dll
 0002:000000ac       __imp___register_onexit_function 004020ac     ucrt:api-ms-win-crt-runtime-l1-1-0.dll
 0002:000000b0       __imp___initialize_onexit_table 004020b0     ucrt:api-ms-win-crt-runtime-l1-1-0.dll
 0002:000000b4       __imp___c_exit             004020b4     ucrt:api-ms-win-crt-runtime-l1-1-0.dll
 0002:000000b8       \177api-ms-win-crt-runtime-l1-1-0_NULL_THUNK_DATA 004020b8     ucrt:api-ms-win-crt-runtime-l1-1-0.dll
 0002:000000bc       __imp____acrt_iob_func     004020bc     ucrt:api-ms-win-crt-stdio-l1-1-0.dll
 0002:000000c0       __imp___set_fmode          004020c0     ucrt:api-ms-win-crt-stdio-l1-1-0.dll
 0002:000000c4       __imp____stdio_common_vfprintf 004020c4     ucrt:api-ms-win-crt-stdio-l1-1-0.dll
 0002:000000c8       __imp____p__commode        004020c8     ucrt:api-ms-win-crt-stdio-l1-1-0.dll
 0002:000000cc       \177api-ms-win-crt-stdio-l1-1-0_NULL_THUNK_DATA 004020cc     ucrt:api-ms-win-crt-stdio-l1-1-0.dll
 0002:000000d0       __imp__JLI_GetStdArgc      004020d0     jli:jli.dll
 0002:000000d4       __imp__JLI_GetStdArgs      004020d4     jli:jli.dll
 0002:000000d8       __imp__JLI_Launch          004020d8     jli:jli.dll
 0002:000000dc       __imp__JLI_MemAlloc        004020dc     jli:jli.dll
 0002:000000e0       __imp__JLI_CmdToArgs       004020e0     jli:jli.dll
 0002:000000e4       \177jli_NULL_THUNK_DATA    004020e4     jli:jli.dll
 0002:000000e8       ___guard_check_icall_fptr  004020e8     MSVCRT:guard_support.obj
 0002:000000ec       ___castguard_check_failure_os_handled_fptr 004020ec     MSVCRT:guard_support.obj
 0002:000000f0       ___xc_a                    004020f0     MSVCRT:initializers.obj
 0002:000000f8       ___xc_z                    004020f8     MSVCRT:initializers.obj
 0002:000000fc       ___xi_a                    004020fc     MSVCRT:initializers.obj
 0002:00000108       ___xi_z                    00402108     MSVCRT:initializers.obj
 0002:0000010c       ___xp_a                    0040210c     MSVCRT:initializers.obj
 0002:00000110       ___xp_z                    00402110     MSVCRT:initializers.obj
 0002:00000114       ___xt_a                    00402114     MSVCRT:initializers.obj
 0002:00000118       ___xt_z                    00402118     MSVCRT:initializers.obj
 0002:00000120       ??_C@_04EFFPLJGM@java@     00402120     main.obj
 0002:00000128       ??_C@_07EBOEHGIC@?9J?9ms8m@ 00402128     main.obj
 0002:00000130       ??_C@_0CN@FOKNIOKM@?9J?9Dsun?4jvm?4hotspot?4debugger?4us@ 00402130     main.obj
 0002:00000160       ??_C@_0CP@KGIPAOBA@?9J?9Dsun?4jvm?4hotspot?4debugger?4us@ 00402160     main.obj
 0002:00000190       ??_C@_0BE@CIMKGGBN@sun?4tools?4jmap?4JMap@ 00402190     main.obj
 0002:000001a4       ??_C@_0P@MAEHPKDA@?1lib?1tools?4jar@ 004021a4     main.obj
 0002:000001b4       ??_C@_0BA@OONPJHCB@?1lib?1sa?9jdi?4jar@ 004021b4     main.obj
 0002:000001c4       ??_C@_08BIJCENIG@?1classes@ 004021c4     main.obj
 0002:000001d0       ??_C@_07JMAJNDJI@openjdk@  004021d0     main.obj
 0002:000001e0       ??_C@_0BF@FJHGBKOC@_JAVA_LAUNCHER_DEBUG@ 004021e0     main.obj
 0002:000001f8       ??_C@_0BN@NGFJBAGH@Windows?5original?5main?5args?3?6@ 004021f8     main.obj
 0002:00000218       ??_C@_0BE@OCLPFDNJ@wwwd_args?$FL?$CFd?$FN?5?$DN?5?$CFs?6@ 00402218     main.obj
 0002:0000022c       ??_C@_03LDGAGIDG@1?48@     0040222c     main.obj
 0002:00000230       ??_C@_0CA@EAHLAFDB@1?48?40_472?9beta?9202510232003?9b08@ 00402230     main.obj
 0002:00000258       __load_config_used         00402258     MSVCRT:loadcfg.obj
 0002:00000380       ___safe_se_handler_table   00402380     <linker-defined>
 0002:00000384       ___volatile_metadata       00402384     <linker-defined>
 0002:000006fc       ___rtc_iaa                 004026fc     MSVCRT:initsect.obj
 0002:00000700       ___rtc_izz                 00402700     MSVCRT:initsect.obj
 0002:00000704       ___rtc_taa                 00402704     MSVCRT:initsect.obj
 0002:00000708       ___rtc_tzz                 00402708     MSVCRT:initsect.obj
 0002:0000074c       __IMPORT_DESCRIPTOR_jli    0040274c     jli:jli.dll
 0002:00000760       __IMPORT_DESCRIPTOR_KERNEL32 00402760     kernel32:KERNEL32.dll
 0002:00000774       __IMPORT_DESCRIPTOR_VCRUNTIME140 00402774     vcruntime:VCRUNTIME140.dll
 0002:00000788       __IMPORT_DESCRIPTOR_api-ms-win-crt-stdio-l1-1-0 00402788     ucrt:api-ms-win-crt-stdio-l1-1-0.dll
 0002:0000079c       __IMPORT_DESCRIPTOR_api-ms-win-crt-runtime-l1-1-0 0040279c     ucrt:api-ms-win-crt-runtime-l1-1-0.dll
 0002:000007b0       __IMPORT_DESCRIPTOR_api-ms-win-crt-environment-l1-1-0 004027b0     ucrt:api-ms-win-crt-environment-l1-1-0.dll
 0002:000007c4       __IMPORT_DESCRIPTOR_api-ms-win-crt-math-l1-1-0 004027c4     ucrt:api-ms-win-crt-math-l1-1-0.dll
 0002:000007d8       __IMPORT_DESCRIPTOR_api-ms-win-crt-locale-l1-1-0 004027d8     ucrt:api-ms-win-crt-locale-l1-1-0.dll
 0002:000007ec       __IMPORT_DESCRIPTOR_api-ms-win-crt-heap-l1-1-0 004027ec     ucrt:api-ms-win-crt-heap-l1-1-0.dll
 0002:00000800       __NULL_IMPORT_DESCRIPTOR   00402800     jli:jli.dll
 0003:00000024       ___scrt_native_dllmain_reason 00403024     MSVCRT:utility.obj
 0003:00000028       ___scrt_default_matherr    00403028     MSVCRT:matherr.obj
 0003:00000030       ___isa_enabled             00403030     MSVCRT:cpu_disp.obj
 0003:00000034       ___security_cookie_complement 00403034     MSVCRT:gs_cookie.obj
 0003:00000038       ___security_cookie         00403038     MSVCRT:gs_cookie.obj
 0003:0000003c       ___scrt_ucrt_dll_is_in_use 0040303c     MSVCRT:ucrt_stubs.obj
 0003:00000040       ___scrt_current_native_startup_state 00403040     MSVCRT:utility.obj
 0003:00000044       ___scrt_native_startup_lock 00403044     MSVCRT:utility.obj
 0003:00000068       ?__type_info_root_node@@3U__type_info_node@@A 00403068     MSVCRT:tncleanup.obj
 0003:00000070       ?_OptionsStorage@?1??__local_stdio_scanf_options@@9@4_KA 00403070     MSVCRT:default_local_stdio_options.obj
 0003:00000078       ___scrt_debugger_hook_flag 00403078     MSVCRT:utility_desktop.obj
 0003:0000007c       ___isa_available           0040307c     MSVCRT:cpu_disp.obj
 0003:00000080       ___favor                   00403080     MSVCRT:cpu_disp.obj
 0003:000003a8       ?_OptionsStorage@?1??__local_stdio_printf_options@@9@9 004033a8     <common>
 0003:000003b0       ___dyn_tls_dtor_callback   004033b0     <common>
 0003:000003b4       ___dyn_tls_init_callback   004033b4     <common>

 entry point at        0001:00000384

 Static symbols

 0000:ffffa000       .debug$S                   00400000     vcruntime:VCRUNTIME140.dll
 0000:ffffa000       .debug$S                   00400000     vcruntime:VCRUNTIME140.dll
 0000:ffffa000       .debug$S                   00400000     vcruntime:VCRUNTIME140.dll
 0000:ffffa000       .debug$S                   00400000     vcruntime:VCRUNTIME140.dll
 0000:ffffa000       .debug$S                   00400000     vcruntime:VCRUNTIME140.dll
 0000:ffffa000       .debug$S                   00400000     ucrt:api-ms-win-crt-environment-l1-1-0.dll
 0000:ffffa000       .debug$S                   00400000     ucrt:api-ms-win-crt-heap-l1-1-0.dll
 0000:ffffa000       .debug$S                   00400000     ucrt:api-ms-win-crt-locale-l1-1-0.dll
 0000:ffffa000       .debug$S                   00400000     ucrt:api-ms-win-crt-math-l1-1-0.dll
 0000:ffffa000       .debug$S                   00400000     ucrt:api-ms-win-crt-runtime-l1-1-0.dll
 0000:ffffa000       .debug$S                   00400000     ucrt:api-ms-win-crt-runtime-l1-1-0.dll
 0000:ffffa000       .debug$S                   00400000     ucrt:api-ms-win-crt-runtime-l1-1-0.dll
 0000:ffffa000       .debug$S                   00400000     ucrt:api-ms-win-crt-runtime-l1-1-0.dll
 0000:ffffa000       .debug$S                   00400000     ucrt:api-ms-win-crt-runtime-l1-1-0.dll
 0000:ffffa000       .debug$S                   00400000     ucrt:api-ms-win-crt-runtime-l1-1-0.dll
 0000:ffffa000       .debug$S                   00400000     ucrt:api-ms-win-crt-runtime-l1-1-0.dll
 0000:ffffa000       .debug$S                   00400000     ucrt:api-ms-win-crt-runtime-l1-1-0.dll
 0000:ffffa000       .debug$S                   00400000     ucrt:api-ms-win-crt-runtime-l1-1-0.dll
 0000:ffffa000       .debug$S                   00400000     ucrt:api-ms-win-crt-runtime-l1-1-0.dll
 0000:ffffa000       .debug$S                   00400000     ucrt:api-ms-win-crt-runtime-l1-1-0.dll
 0000:ffffa000       .debug$S                   00400000     ucrt:api-ms-win-crt-runtime-l1-1-0.dll
 0000:ffffa000       .debug$S                   00400000     ucrt:api-ms-win-crt-runtime-l1-1-0.dll
 0000:ffffa000       .debug$S                   00400000     ucrt:api-ms-win-crt-runtime-l1-1-0.dll
 0000:ffffa000       .debug$S                   00400000     ucrt:api-ms-win-crt-runtime-l1-1-0.dll
 0000:ffffa000       .debug$S                   00400000     ucrt:api-ms-win-crt-runtime-l1-1-0.dll
 0000:ffffa000       .debug$S                   00400000     ucrt:api-ms-win-crt-runtime-l1-1-0.dll
 0000:ffffa000       .debug$S                   00400000     ucrt:api-ms-win-crt-runtime-l1-1-0.dll
 0000:ffffa000       .debug$S                   00400000     ucrt:api-ms-win-crt-runtime-l1-1-0.dll
 0000:ffffa000       .debug$S                   00400000     ucrt:api-ms-win-crt-runtime-l1-1-0.dll
 0000:ffffa000       .debug$S                   00400000     ucrt:api-ms-win-crt-runtime-l1-1-0.dll
 0000:ffffa000       .debug$S                   00400000     ucrt:api-ms-win-crt-runtime-l1-1-0.dll
 0000:ffffa000       .debug$S                   00400000     ucrt:api-ms-win-crt-stdio-l1-1-0.dll
 0000:ffffa000       .debug$S                   00400000     ucrt:api-ms-win-crt-stdio-l1-1-0.dll
 0000:ffffa000       .debug$S                   00400000     ucrt:api-ms-win-crt-stdio-l1-1-0.dll
 0000:ffffa000       .debug$S                   00400000     ucrt:api-ms-win-crt-stdio-l1-1-0.dll
 0000:ffffa000       .debug$S                   00400000     kernel32:KERNEL32.dll
 0000:ffffa000       .debug$S                   00400000     kernel32:KERNEL32.dll
 0000:ffffa000       .debug$S                   00400000     kernel32:KERNEL32.dll
 0000:ffffa000       .debug$S                   00400000     kernel32:KERNEL32.dll
 0000:ffffa000       .debug$S                   00400000     kernel32:KERNEL32.dll
 0000:ffffa000       .debug$S                   00400000     kernel32:KERNEL32.dll
 0000:ffffa000       .debug$S                   00400000     kernel32:KERNEL32.dll
 0000:ffffa000       .debug$S                   00400000     kernel32:KERNEL32.dll
 0000:ffffa000       .debug$S                   00400000     kernel32:KERNEL32.dll
 0000:ffffa000       .debug$S                   00400000     kernel32:KERNEL32.dll
 0000:ffffa000       .debug$S                   00400000     kernel32:KERNEL32.dll
 0000:ffffa000       .debug$S                   00400000     kernel32:KERNEL32.dll
 0000:ffffa000       .debug$S                   00400000     kernel32:KERNEL32.dll
 0000:ffffa000       .debug$S                   00400000     kernel32:KERNEL32.dll
 0000:ffffa000       .debug$S                   00400000     jli:jli.dll
 0000:ffffa000       .debug$S                   00400000     jli:jli.dll
 0000:ffffa000       .debug$S                   00400000     jli:jli.dll
 0000:ffffa000       .debug$S                   00400000     jli:jli.dll
 0000:ffffa000       .debug$S                   00400000     jli:jli.dll
 0001:0000013d       ?pre_c_initialization@@YAHXZ 0040113d f   MSVCRT:exe_main.obj
 0001:000001e8       ?post_pgo_initialization@@YAHXZ 004011e8 f   MSVCRT:exe_main.obj
 0001:000001f0       ?pre_cpp_initialization@@YAXXZ 004011f0 f   MSVCRT:exe_main.obj
 0001:00000202       ?__scrt_common_main_seh@@YAHXZ 00401202 f   MSVCRT:exe_main.obj
 0001:0000038e       ?find_pe_section@@YAPAU_IMAGE_SECTION_HEADER@@QAEI@Z 0040138e f   MSVCRT:utility.obj
 0001:000005df       ___get_entropy             004015df f   MSVCRT:gs_support.obj
 0001:00000920       $$000000                   00401920     MSVCRT:sehprolg4.obj
 0002:000000f4       ?pre_cpp_initializer@@3P6AXXZA 004020f4     MSVCRT:exe_main.obj
 0002:00000100       ?pre_c_initializer@@3P6AHXZA 00402100     MSVCRT:exe_main.obj
 0002:00000104       ?post_pgo_initializer@@3P6AHXZA 00402104     MSVCRT:exe_main.obj
 0002:000001d8       _const_cpwildcard          004021d8     main.obj
 0002:000001dc       _const_ergo_class          004021dc     main.obj
 0002:00000250       _GS_ExceptionPointers      00402250     MSVCRT:gs_report.obj
 0002:00000710       __sehtable$?__scrt_common_main_seh@@YAHXZ 00402710     MSVCRT:exe_main.obj
 0002:00000730       __sehtable$___scrt_is_nonwritable_in_current_image 00402730     MSVCRT:utility.obj
 0002:0000094e       .idata$6                   0040294e     jli:jli.dll
 0002:00000a84       .idata$6                   00402a84     kernel32:KERNEL32.dll
 0002:00000aea       .idata$6                   00402aea     vcruntime:VCRUNTIME140.dll
 0002:00000cf4       .idata$6                   00402cf4     ucrt:api-ms-win-crt-stdio-l1-1-0.dll
 0002:00000d14       .idata$6                   00402d14     ucrt:api-ms-win-crt-runtime-l1-1-0.dll
 0002:00000d36       .idata$6                   00402d36     ucrt:api-ms-win-crt-environment-l1-1-0.dll
 0002:00000d5c       .idata$6                   00402d5c     ucrt:api-ms-win-crt-math-l1-1-0.dll
 0002:00000d7c       .idata$6                   00402d7c     ucrt:api-ms-win-crt-locale-l1-1-0.dll
 0002:00000d9e       .idata$6                   00402d9e     ucrt:api-ms-win-crt-heap-l1-1-0.dll
 0003:00000000       _const_progname            00403000     main.obj
 0003:00000004       _const_jargs               00403004     main.obj
 0003:00000014       _const_appclasspath        00403014     main.obj
 0003:00000020       _const_launcher            00403020     main.obj
 0003:00000048       ?is_initialized_as_dll@@3_NA 00403048     MSVCRT:utility.obj
 0003:00000049       ?module_local_atexit_table_initialized@@3_NA 00403049     MSVCRT:utility.obj
 0003:0000004c       ?module_local_atexit_table@@3U_onexit_table_t@@A 0040304c     MSVCRT:utility.obj
 0003:00000058       ?module_local_at_quick_exit_table@@3U_onexit_table_t@@A 00403058     MSVCRT:utility.obj
 0003:00000088       _GS_ExceptionRecord        00403088     MSVCRT:gs_report.obj
 0003:000000d8       _GS_ContextRecord          004030d8     MSVCRT:gs_report.obj
 0004:00000060       $R000000                   00404060     jmap.exe.res
